:060000000C946D010C944C
:100006009D0B0C9400000C9400000C9400000C94C2
:1000160000000C9400000C9400000C9400000C945A
:1000260000000C942D020C9400000C9400000C941B
:1000360000000C9400000C9400000C9404020C9434
:1000460000000C94FA080C9400000C9446090C94D9
:1000560000000C9400000C9400000C9400000C941A
:1000660000000C9400000C9400000C9400000C940A
:1000760000000C94700A0C9400000C94540B0C9421
:1000860000000C94000000010204081020408000CB
:1000960068010000801002006C01150001100000CC
:1000A6007A01130001010000820101000102000033
:1000B6008C0102000102000096010300010200000B
:1000C600A001040001020000AA01050001020000CF
:1000D600B401060001020000BE0107000102000093
:1000E600C801080001020000D20109000102000057
:1000F600DC010A0001020000E6010B00010200001B
:10010600F0010C0001020000FA010D0001020000DE
:1001160004020E00010200000E020F0001020000A0
:100126001802100001020000220211000102000064
:100136002C0212000102000000000000FF00000077
:10014600000001000200040008001000200040002A
:10015600800000010002000400080010002000409A
:1001660000805F4944005F53656E64496E70757424
:10017600546F00005F52656C616973005F496E7071
:1001860075745F3100005F496E7075745F320000F0
:100196005F496E7075745F3300005F496E707574E9
:1001A6005F3400005F496E7075745F3500005F490B
:1001B6006E7075745F3600005F496E7075745F37D8
:1001C60000005F496E7075745F3800005F496E709D
:1001D60075745F3900005F496E7075745F31300069
:1001E6005F496E7075745F3131005F496E7075746A
:1001F6005F3132005F496E7075745F3133005F495D
:100206006E7075745F3134005F496E7075745F315E
:1002160035005F496E7075745F3136005F496E70E8
:1002260075745F3137005F496E7075745F313800E1
:100236001027E80364000A00010000100001100006
:10024600010049530049430025642E2532640044C9
:100256005300564300494C00235022415343494919
:100266002D492F4F222C22312E3030222C32303085
:10027600382D30312D30313B0023482245636F2223
:100286002C22312E3030222C323030382D30312D88
:1002960030313B0023532245636F222C22312E300E
:1002A60030222C323030382D30312D30313B0000A9
:1002B600256400253032580025313064000056434D
:1002C6000049500001002D4E414E00000100E00F94
:1002D600CA020000F894EE27ECBBF1E0F5BFE5BFDB
:1002E600E0936C00F8E1F1BDE1BD8DE0A2E0BB2733
:1002F600ED938A95E9F780E090E1A0E0B1E0ED9317
:100306000197E9F7E2EDF2E085919591009761F0AA
:10031600A591B59105901590BF01F00105900D923C
:100326000197E1F7FB01F0CFEFEFEDBFE0E1EEBFA4
:10033600C0E0D5E00C946B03E0916300E071089592
:10034600E881E03011F01A9801C01A9A0C94EE0474
:100356001A930A930E943F1300000000000009B39D
:1003660011270E944913000000000000E9B3FE2F88
:10037600E0E00E0F1F1FE0EEE5BBEFEFEABB0C94CB
:100386004704F8940E943F13000000000000E9B300
:10039600E093920B0E944913000000000000A3E9BD
:1003A600BBE0E9B3EC93E0EEE5BBEFEFEABB789494
:1003B6000895F894A091DF0CB091E00CEFEFF0E017
:1003C600EA27FB27EBBBE0ECE5BBE0EEE5BB000074
:1003D600E091DF0CF091E00C0E94C015AFEFB0E0A9
:1003E600EA27FB27EBBBE0EAE5BBE0EEE5BB000056
:1003F6000E943F04E87011F4C79A01C0C798789428
:1004060008950E945113E4E6E2BF0E94180478940E
:100416004394E2E3E41519F4E1E0E71509F002C0BC
:1004260077244424E2E3E41519F4E0E0E71509F043
:1004360003C0E1E07E2E4424A0910105A13028F0FE
:10044600E0910105E150E09301059BDF0E94BB0EA0
:10045600B0DF0BC00E945113E6E0E4BD79DFFA93EA
:10046600EA930E942E0E0E94E10DE991EFBFF991E9
:10047600E991B991A9919991899179916991F990A7
:100486001990099018951A93A0915808A13051F423
:10049600DA92CA92E4E6F0E0FA93EA930E944B04F9
:1004A600E03009F409C0E0E0E0935808E3E0E9151C
:1004B60018F40E945F139924A0915808A23041F4C1
:1004C600DA92CA920E9467130E944B04E03009F444
:1004D60003C0E0E0E0935808A0915808A03059F412
:1004E600E0915106A0915206EA1729F0A0E020FCFF
:1004F600A1E0A03009F027C00E946C13EE5FFA4F0E
:10050600E081E13039F40E946C130E9472130E945C
:10051600791319C0E23011F0E330A9F40E946C138C
:10052600EE5FFA4FE081E23009F499240E946C13E1
:100536000E947213EE5FFA4FA3E0A0839DD16F0174
:10054600E1E0E09358080C9417051A93A09155061C
:10055600A43011F410918A07A0915506A53011F424
:100566001091F107143049F4E981E03011F4E0E02C
:1005760001C0EFE0EA930E949704153049F4E9813F
:10058600E03011F4E5E101C0E6E0EA930E94970449
:1005960062C01A93E3E0EA930E949704109154060E
:1005A600E12FE295EF700E947E13E12FEF700E941B
:1005B6007E13E7E1EA930E9497040C941705E2E0A4
:1005C600EA930E949704E0E0E0935406E9E4EA9394
:1005D6000E949704E881E05DEA930E949704D9DFC0
:1005E600A0915506A43011F40E9484130E948B1327
:1005F6001696E1E0EC93E8810E9490130C94EE04C9
:100606001A93A0915506A43011F40E94841310E0A9
:10061600173060F40E948B131A96EE27A10FBE1FA7
:10062600EC91EA930E9497041F5FF2CFE981E030D4
:1006360011F4E0E305C0E091060DF091070DE189A4
:10064600EA930E9497040E948B131696E1E0EC93BE
:10065600E9810E949013188122960895E091590627
:10066600A0915806EA1761F0A0915706A13041F40F
:100676000E943509EB3020F00E949F01E03009F41A
:100686000FC0E0915906F0E0E65AF94FE081EA938F
:100696000E947609A09159060E949713E093590685
:1006A60008951A93A8950E94520D0E941C0DEBDE28
:1006B600D5DFE0E0E71521F4A0910105A03011F0A7
:1006C600E1E001C0E0E0EA930E94A3010C94170563
:1006D600E0E0E5BFE0936D00E0936C00EFEFEBBB6D
:1006E600EABBE5BBE4BBE0E0E2BBE1BBE093620052
:1006F600E0936100ECE9E3B9E2B9E7E0E093650075
:10070600E0936400EFE0E8BBE0E8E7BBE0E0E0BFD1
:10071600E7E0E3BFE4E6E2BFE0E0E1BFEFBDEEBD48
:10072600EDBDECBDE7BDE6BDEBBDEABDE9BDE8BD8F
:10073600E0937900E0937800E3E0E5BDE6E0E4BD10
:10074600E0E0E3BDE0938B00EAE0E0938A00E0E0BE
:10075600E0938900E0938800E0938100E0938000B5
:10076600E2E1E0938700E4E3E0938600E0E0E093D3
:100776008500E0938400E0938300E0938200E09399
:100786006A00EABFE9BFE1E4E7BFE0E0E0937D008D
:10079600EBB9E8EDEAB9E6E0E0939500E0E0E09336
:1007A6009000E6E6E9B9E0E0E0939B00E8EDE0932F
:1007B6009A00E6E0E0939D00E0E0E0939800E3E332
:1007C600E0939900E0E8E8B9E0E0E0BDEEE1E1BDE4
:1007D600EEE0E1BD0E94D5080E9428110E949C13FC
:1007E600E53128F0A0E0B0E0E0E00E944816A895C8
:1007F6000E94A11388240E949C138E1648F4A89583
:10080600E1E00E94A713E0E00E94A7138394F3CFD0
:100816000E94A1137894EFEF6E2E43DF0E94EC1036
:10082600E1E0E0935706F9CFFFCFA8E0BDE00E94D4
:10083600B0130895A881A03310F0AA3308F003C0BE
:10084600E881E053C8C0A881A13410F0A73408F0AD
:1008560003C0E881E753BFC0EFEFBDC0A881AA304F
:1008660018F4E881E05DB7C0A881AA3018F0E881E5
:10087600E95CB1C0E8E5AFC01A930A93F894009119
:10088600080D1091090D7894F801099119910895B0
:100896001A930A93F1DF8F01EA81FB81AC81BD8156
:1008A600EA0FFB1FE01BF10BDF010E94591624F42F
:1008B600E0E019810881E9C2E1E019810881E5C219
:1008C600E881EF5FE883A881A53010F0E0E0E883D7
:1008D600E88181C0A0915206BB27E0915106F0E065
:1008E60031960E94B6133596DF01E5E0F0E00C94F0
:1008F6004309A0915906BB27E09158060C943A0982
:10090600A0915306A13059F4A0915706A13039F4AD
:10091600F0DFE93220F00E949F01E03009F402C0C6
:10092600E1E00895E0E00895E881A0915406EA2701
:10093600E0935406E0915506E13071F4E0915806D3
:10094600F0E0E65AF94FA881A083A09158060E94CC
:100956009713E09358063FC0E23071F4E091BE066B
:10096600F0E0E054F94FA881A083A091BE060E9452
:100976009713E093BE062FC0E33071F4E09124078D
:10098600F0E0EA5DF84FA881A083A09124070E94B9
:100996009713E09324071FC0E43071F4E0918B07AE
:1009A600F0E0E357F84FA881A083A0918B070E943F
:1009B6009713E0938B070FC0E53069F4E091F207D7
:1009C600F0E0EC50F84FA881A083A091F2070E94B6
:1009D6009713E093F20721960895E0915C0BEA9352
:1009E6000E94380CE0915D0BEA930E94380C089542
:1009F600F4DF0E94BB130E94BB13E881F9810E94B9
:100A0600C5130C949D091A930E940C0C1E2F1030CE
:100A160021F0E12FE150E0935B0BDFDFE0915B0B10
:100A2600EF5FF0E00E94C5131991089528970E9480
:100A36005D1650E00E94CF0BE13010F40C946B066B
:100A4600E0915C0BE43411F00C949A05E0915D0B97
:100A5600E33221F40E940C0CE0935306E0915D0B07
:100A6600E33549F4E5E5F2E00E94CD1349DFE05DA8
:100A7600EA930E94380CE0915D0BE03511F00C947E
:100A86009905E2E2EA930E94C30BE03019F0AF85C4
:100A9600A13009F04BC020E00E94D113A03240F0F3
:100AA6000E94D113A23221F00E94D113AB3309F474
:100AB6003DC0E22FE03071F40E94D113A33211F44D
:100AC60021E007C0E0915306E09355060E94D71334
:100AD6002BDF29C0E13049F40E94D113A43211F46E
:100AE60022E001C020E010E01EC0E23011F0E33049
:100AF600D1F40E94D7139EDEEF3FA1F0E12FE295DD
:100B0600E07F4E2F0E94D71395DEE40F1E2F2F5F36
:100B1600243039F4E0915306E09355061A9304DF26
:100B260020E001C020E00E94DE13B6CFCEC0E6353D
:100B360011F00C944F06E0915D0BE334B1F50E9481
:100B4600E11330E0303188F50E94E713E156F44FA7
:100B5600E0811E1741F5AFEDBBE0EE27A30FBE1FE8
:100B6600AC91A230D9F4E8E5F2E00E94CD13E12F72
:100B76000E94EA130E94F013AFE4BCE00E94E71360
:100B86000E94F4130E94FB130E94F013AFE6BCE030
:100B96000E94E7130E94F4130E94C5130E94E713F4
:100BA6000E94FF1302C03F5FCDCFE0915D0BE3359E
:100BB60011F00C941F060E940C0CE093970B0E94F8
:100BC6000414C9F50E940C0CE093980B0E940414BF
:100BD60091F50E940C0CE093990BE03019F0E1E0DE
:100BE600E093990B0E94041431F50E940C0CE093DB
:100BF6009B0BF0939C0B0E940414E9F40E940C0CCE
:100C0600E0939D0BF0939E0B0E940414A1F40E94A6
:100C1600E113EE85E0939A0BE0E0EA931A930E94C3
:100C2600F40FE03041F4E8E5F2E00E94CD130E94B3
:100C36000A140E94C51349C0E0915D0BE53559F5CC
:100C46000E94E1130E94041429F50E940C0C0E2F39
:100C560030E03031F8F40E94E713E156F44FE081BA
:100C66001E17B1F4013049F4AFECBBE00E94E71364
:100C76000E940D14E068D001EC93003049F4AFEC0B
:100C8600BBE00E94E7130E940D14EF77D001EC93AE
:100C96003F5FDFCF1AC019C0E934B9F4E0915D0BAC
:100CA600EC3499F4EBE5F2E00E94CD13E091920B5F
:100CB6000E941714E091930B0E941714E091940B75
:100CC600F0E0FA93EA930E94760C0E94B00BB2CE43
:100CD6000E941D14609608950E945D160E94CF0B17
:100CE600E13010F40C944607E0915C0BE33211F509
:100CF600E0915D0BEC3431F4E4E0E093E10CE0E0EC
:100D0600E093760BE0915D0BE43599F4E091760B78
:100D1600E03029F0EF77A0E0B0E00E9448160E948C
:100D260067130E94A515E0E0E093760BE7E0E093F9
:100D3600E10C04C0E43511F00C944307E0915D0B1F
:100D4600E33231F40E940C0C3197E0935B0B98C0B0
:100D5600E03511F00C94430710E00E94D113A03245
:100D660050F00E94D113AD3331F00E94D113AB3352
:100D760011F01E3008F00CC00E940A14E25AF44F1B
:100D86000E942614D001EC931F5F0E94DE13E5CF6C
:100D96000E940A14E25AF44FA0E0A083EDE3EA931E
:100DA6000E94C30BE13011F00C944307E4E5E09395
:100DB600720B10E00E940A140E942D143496E491DE
:100DC600EF3F11F40C9443070E9432140E940A1458
:100DD6000E942D140E942016FA93EA930E948E1107
:100DE600E03011F00C9441070E940A140E942D1461
:100DF6003496E491E03839F40E940C0CE058FF4F29
:100E0600E093760B3BC0E03011F0E130A1F40E9494
:100E16000A140E942D1432960E942016FF93EF9317
:100E26000E940C0CAF91BF910E9448160E94671356
:100E36000E94A51523C0E23081F40E940A140E9484
:100E46002D1432960E942016FF93EF930E940C0CED
:100E5600AF91BF910E94401611C0E33079F40E9411
:100E66000A140E942D1432960E942016FF93EF93C7
:100E76000E94EB0BAF91BF910E9448161F5F9ACF5D
:100E86000E94B00B2BCF0E941D14269608950E9437
:100E96005F160E94CF0BE13010F40C94BF07E0916F
:100EA6005C0BE332A9F4E0915D0BE03519F4EEE555
:100EB600F2E009C0E83419F4EFE7F2E004C0E335E4
:100EC60031F4EAE9F2E0FA93EA930E94490C51C040
:100ED600E43511F00C94BC07E0915D0BE43231F47B
:100EE600E5E1F0E0FA93EA9383DD43C0E33211F4DF
:100EF6008ADD3FC0E035E9F570DDA0915B0BA531D9
:100F0600C0F50E9437140E9420160E94CD13EDE30F
:100F1600EA930E94380C0E9437143496E491E03824
:100F260029F40E949C130E943B1423C0E03011F068
:100F3600E13049F40E9437140E943D140E94341691
:100F46000E943B1416C0E23049F40E9437140E94F6
:100F56003D140E9430160E94FB130BC0E33049F487
:100F66000E9437140E943D140E943416EA930E9490
:100F7600840C0E94B00B8DCF0E944214E0E0EC93EB
:100F86000E946616249608951A930A9300E0A0918B
:100F96005808A13081F40E946C13EE5FFA4FE0818D
:100FA600E33049F40E946C13EB5FFA4FE381A091A2
:100FB6005E0AEA1709F03FC00E94471401E00E944A
:100FC600CF0BE130A0F1E0915C0BE23479F5E091D2
:100FD6005D0BE13459F50E940C0C1E2F0E946C1318
:100FE600ED5FFA4FE081E09355060E946C13EC5FCB
:100FF600FA4FE081E73419F41A930E94A8020E947E
:101006006C13EC5FFA4FE081E33419F41A930E94F3
:10101600E2020E946C13EC5FFA4FE081E53419F4AA
:101026001A930E940303EEE1E0930105C8CF0E94E4
:101036006C130E947913E02F0C94090C1A930A93EF
:101046000E94471447DCE23078F10E944E140E9459
:1010560054140E9461140E944214E2E70E9468142C
:10106600E0915E0A0E946C140E946E14A0915E0AC2
:10107600E0910A0DEA1721F4E0915E0AE03311F4DB
:1010860001E001C000E0E0915E0AE0930A0D0A93D8
:10109600E0915C0AEA93CADC0E9471140E944E1425
:1010A6000E9475140C94090CE0E00C94090C1A9338
:1010B600EBE5F9E00E948214EBE5F8E00E94871464
:1010C6000E9471140E948C14E181E43471F40E9430
:1010D6008C1402800E949C13E05DE01529F00E94AA
:1010E6008C14E281EA3209F401C028C00E949114EE
:1010F6000E948C14E1810E946C140E948C14E2817F
:101106000E946C140E9494141C910E948C143396B5
:101116000E948714E12FE23139F40E94421413979A
:10112600E6E0EC93D9DD08C0E13131F40E944214C7
:101136001397E2E1EC93ABDE0E94A00C0C94680CD2
:101146001A93C8DBE23058F10E944E140E945414E0
:101156000E9461140E944214EAE70E946814EFE5B7
:10116600FAE00E9487140E94941411971C91E12FB3
:10117600E23131F4E6E0EA930E94380CADDD07C0B7
:10118600E13129F4E2E1EA930E94380C80DE0E9404
:1011960071140E944E140E9475140C94680CE0E0C1
:1011A6000C94680CEFEFE093720BE093730B0895C9
:1011B600AC81A03310F0AA3308F006C00E9499143F
:1011C600E0530E94A1140FC0AC81A13410F0A734E3
:1011D60008F006C00E949914E7530E94A11403C0A8
:1011E600A881B981E0E0EC9325960895EDC2AA9313
:1011F600EA93FA93EFB7EA931A930A931BB10CB1E9
:10120600E0914A0DF0E0E85EF24F0083A0914A0DAE
:10121600AF5FA0934A0DA23319F4E0E0E0934A0DC4
:10122600099119915CC21A93E0914B0DA0914A0D58
:10123600EA17D1F3F0E0E85EF24F1081A0914B0D72
:10124600AF5FA0934B0DA23319F4E0E0E0934B0D92
:10125600E12F3BC3E0914B0DA0914A0DEA1709F02F
:10126600B3C2B4C2A091B10DBB27E091B00DF0E0BE
:1012760031960E94B613EC59FF4FDF01E4E6F0E029
:101286000E94001608950E945113E091B10DA0919D
:10129600B00DEA1741F0A0915706A03019F0A6DF6D
:1012A600E03009F001C011C0E091B10DF0E0E45B5F
:1012B600F24FE081ECB9A091B10DAF5FA093B10DF3
:1012C600A43619F4E0E0E093B10DE991EFBFF9918E
:1012D600E991B991A9919991899179916991F99039
:1012E6001990099018951A93E091B10DA091B00D3F
:1012F600EA1751F45D9B08C0A0915706A13019F476
:1013060075DFE03009F013C01091B00D0E940A1489
:10131600E45BF24FA981A0831F5F143609F410E045
:10132600E091B10DE117E1F31093B00D02C0E98130
:10133600ECB91881229608950E945F168BDFE03083
:1013460021F0A0915A08A03009F0C6C06CDF1E2F0C
:10135600A091160DA53618F0E0E0E093120D30913D
:10136600120DE091120DE03059F4113019F4E4E059
:10137600E093120D1A3519F4EBE0E093120DA4C0B8
:10138600E43089F4E0E0E093120D10935B081093CB
:10139600140DE6E0E093120DE0E0E0935A08E1E078
:1013A600E093130D91C0E53091F4E0E0E093120D67
:1013B6000E949C13E05DE11749F00E94AA140E9466
:1013C600B1140E94B814E6E0E093120D7DC0E63039
:1013D60091F40E94B1140E94AA14133049F4E7E074
:1013E600E093120DE0E0E093150D0E94BE1402C0DA
:1013F6000E94B81469C0E73011F0E83059F41A9326
:10140600E5E1FDE0FA93EA93E2E1FDE0FA93EA937F
:10141600CFDE5AC0E93081F4E0E0E093120D1731D7
:1014260031F4E091150DA091140DEA1709F003C0EF
:10143600E4E5E0935A0848C0EB3069F4103039F41B
:10144600ECE0E093120DE0E0E0935A0803C0E0E020
:10145600E093120D39C0EC3049F41093170D109338
:10146600140DE0E0E093130DEDE02CC0ED3011F526
:101476000E94B1140E94B8140E94AA14E091170D9C
:10148600E150E093170DE030A1F4E091140DE03047
:1014960069F4EEE0E093120DE091130DE1500E9425
:1014A600C614A0E0A0830E94BE1403C0E0E0E0934F
:1014B600120D0AC0EE3041F41D3019F4EAE5E0934E
:1014C6005A08E0E0E093120DE091120DE31719F0CF
:1014D600E0E0E093160D32CFDEC2AA93BA93EA9308
:1014E600FA93EFB7EA931A930A9310919B0000912F
:1014F6009C00E12FEC71A9F4E0917A0EF0917B0E3D
:10150600EE54F24F0083AAE7BEE00E94B013E83C17
:10151600A0E0FA0731F4E0E0F0E0E0937A0EF09311
:101526007B0E09911991E991EFBFF991E991B99172
:10153600A99118951A930E94CA140E94CF14D9F340
:101546000E94CA14EE54F24F1081ACE7BEE00E942E
:10155600B013E83CA0E0FA0731F4E0E0F0E0E093F5
:101566007C0EF0937D0EE12FB0C10E94CA140E943A
:10157600CF1409F029C12AC10E945F16F6DFE030B8
:1015860021F0A0910F0DA03009F08AC0D3DF1E2FE5
:10159600A091100DA53618F0E0E0E0930B0D309108
:1015A6000B0DE0910B0DE03031F4113019F4E4E04D
:1015B600E0930B0D6DC0E430C1F4E0E0E0930B0D59
:1015C6001A3229F00E949C13E05DE11769F410932A
:1015D6005B0A10930D0DE5E0E0930B0DE0E0E09360
:1015E6000F0DE1E0E0930C0D53C0E530A9F4E0E007
:1015F600E0930B0D0E949C13E05DE11761F00E94E1
:10160600D6140E94DD14E0910C0DEF5FE0930C0DF3
:10161600E6E0E0930B0D3CC0E630D1F40E94DD1409
:101626000E94D614133071F4E7E0E0930B0DE0E06E
:10163600E0930E0DE0910C0DF0E0E55AF54FA0E0B9
:10164600A08305C0E0910C0DEF5FE0930C0D20C068
:10165600E73011F0E83059F41A93EEE0FDE0FA9322
:10166600EA93EBE0FDE0FA93EA93A2DD11C0E930DC
:1016760079F4E0E0E0930B0D173131F4E0910E0DB3
:10168600A0910D0DEA1709F003C0E4E5E0930F0DF4
:10169600E0910B0DE31719F0E0E0E093100D6ECF2B
:1016A600FAC1AA93EA93FA93EFB7EA93E091810F0E
:1016B600A091800FEA1781F0E0915908E03019F007
:1016C600E89421F808C00E94E4140E94F21419F468
:1016D600E0E0E093810F03C0E89420F821F8E99157
:1016E600EFBFF991E991A9911895E881A091110DA3
:1016F600EA0FE093110DE091800FF0E0E058F14F12
:10170600A881A083E091800FEF5FE093800F0E9495
:10171600F21419F4E0E0E093800FB6C0E0E0E09345
:10172600810FA091800FA13020F00E94E4146894EC
:1017360021F80895AA93BA93EA93EFB7EA93E0E003
:10174600E093810F0E949C13EF5FE0935908E991A3
:10175600EFBFE991B991A99118950E94D113A032D2
:1017660020F00E94D113AB3309F403C00E94DE13AC
:10177600F4CF0E94D113AB3311F40E94DE13089507
:101786000E94D113E881EA1729F40E94DE133197EB
:10179600E1E07AC0E0E078C00E94D113A03228F0E0
:1017A6000E948C14E181E03208F410C00E94941467
:1017B600EC91E0935C0B0E94DE130E949414EC9172
:1017C600E0935D0B0E94DE13E1E00895E0E00895EA
:1017D6001A930A9310E00E9494140C910B3311F0A3
:1017E600003208F412C0013310F0093308F007C0C4
:1017F600E02FE053F0E0E457FF4FE4911E2B0E94E8
:10180600DE130E9494140C91E9CFE12F09911991EE
:1018160008950E945F1600E010E00E94D113AD32D9
:1018260029F40E94DE132FEF3FEF02C021E030E0E3
:101836000E94D113A03320F00E94D113AA3308F0DE
:101846000FC0D801EAE0F0E00E94D2150E942614EB
:10185600E053F0E0E00DF11D8F010E94DE13E8CFAA
:10186600F901D8010E94D21516C1E8810E946C14B4
:10187600E881A091770BEA0FE093770BE881A091BE
:10188600780BEA27E093780B219608951A9310E0D7
:101896000E94F714E03031F00E94F714EA93E5DF76
:1018A6001F5FF6CF2BC01A9310E00E940A14E25A6B
:1018B600F44FE081E03049F00E940A14E25AF44FF6
:1018C600E081EA93D2DF1F5FF0CF199108950E945D
:1018D6003214E6EBF2E0FA93EA93EC81FD810E9482
:1018E600FF140C94E7101A930E943214E9EBF2E00D
:1018F600FA93EA93ED81FE810E94FF1418812396E4
:1019060008951A93ECE3EA93B0DF11E0193080F4FE
:101916000E940A14E457FF4FE491A981EA2319F0C3
:10192600E12FE05D01C0E0E2EA939FDF1F5FEECFAB
:10193600EEE3EA939ADF0C94E6101A930A93E09189
:101946005B09E03011F40C942511EAE5EA93CBDC4F
:10195600E0E0EA93C8DC10E00E940A14E55AF64F6C
:10196600E081E03011F01F5FF7CF1F5F012F0A9370
:10197600BADC10E00E940A14E55AF64FE081E03026
:1019860079F00E940A14E55AF64FE081EA93ABDC3F
:101996000E940A14E55AF64FE0810E0F1F5FEACF48
:1019A600E02FE195EA939FDCEDE0EA939CDC0C9452
:1019B60025110E945F16AC81BD81EC91E03021F4C7
:1019C6000E9466160C948C11E0E0E093800FE1E033
:1019D600EA938BDEE0E0E093110DAC81BD81EC91E2
:1019E600E03041F0EA9381DEEC81FD813196EC83B3
:1019F600FD83F3CFE3E0EA9378DEE091110DE29503
:101A0600EF70EA930E9431040E2FE091110DEF70F2
:101A1600EA930E9431043E2F0A9367DE3A9365DE0D
:101A2600E7E1EA9362DE689420F80E9466160C9459
:101A36008C110E945F1680DCA0915A08AA3511F419
:101A46000E945A08A0915A08A43511F500E00E9498
:101A56004E14EB5FFA4F9F01E02F0E94C614E081FF
:101A6600E03051F0E02F0E94C614E081D901EC93DA
:101A76000F5F2F5F3F4FF0CFD901E0E0EC930E945C
:101A86004E140E940915E0E0E0935A08E12F03C0C6
:101A9600E0E0E0935A080E946616249608950E9494
:101AA6005D166ADDA0910F0DA43511F00C94DE0DC4
:101AB60010E0A0915B0AAA3221F4E0915D0AED34B0
:101AC60009F059C0E7E0E093E10CE0915E0AEA35DF
:101AD60011F00C94B00D00E04FEF5FEFE091600A5B
:101AE600E7703E2FE0915F0AE23361F4A4E1B0E0D3
:101AF6000E943416AE2F0E94E713E457FF4FE4917D
:101B0600EA2309F414C0E1E6FAE00E9487140E9471
:101B1600D113AB3421F40E94DE137BDE0E2F0E941C
:101B2600D113A43521F40E94DE1373DEAF010093B6
:101B36000005E8ECF0E0E093950BF093960B4093EC
:101B4600E50C5093E60CE2E0E093E10CE0915F0ACD
:101B5600E93319F4E1E0E093E10CE0915E0AE03547
:101B660019F4E1E0E093E10CE0915E0AE23419F445
:101B7600E1E0E093E10C0E949C13E05DA0915B0A1A
:101B8600EA1799F4E0915D0AE23521F40E942108F2
:101B96001E2F0BC0E23721F40E94C7071E2F05C077
:101BA600EA3519F40E94A3081E2FE0E0E0930F0D1A
:101BB600E12F0C948A11E0E00C948A11A0E020FC3D
:101BC600A1E0A13049F4A0E021FCA1E0A03021F47D
:101BD600A0915908A03009F001C0A0DDE091590894
:101BE600E03019F0E150E09359080895A881A13139
:101BF60018F0E881E051E883E8810E941515A0916C
:101C0600DC0FB091DD0FEA2BFB2BE093DC0FF0939A
:101C1600DD0F0C94B9111A930A9310E01031D0F429
:101C26000E940A140E94FF13AFEBBBE0EE27A10F40
:101C3600BE1FEC93AFECBBE0EE27A10FBE1FEC93EB
:101C4600AFE0BCE00E940A140E941F150E942415F2
:101C56001F5FE4CFF7C20E945F16E0917D0BF09103
:101C66007E0BAC81BD81EA27FB279F0110E0123174
:101C760090F4F901E17039F0A12FB0E0A058B44F0B
:101C8600EC91EF5FEC93D901E2E0F0E00E94F815E9
:101C96009F011F5FECCFEC81FD81E0937D0BF093FC
:101CA6007E0B0E94661635C30E946D04E03061F11A
:101CB6000E944E14EB5FFA4F0E948214AFEABBE01B
:101CC600E881F0E0AE0FBF1FEC910E946C140E94F9
:101CD6009C13E05D0E946C140E944214E2E50E948F
:101CE60068140E9429150E946E14E4ECF2E00E942A
:101CF600CD13E8810E9435150E94EA130E947114E3
:101D06000E944E140E9409150C94B9110E946D048C
:101D1600E03069F10E944E14EB5FFA4F0E94821484
:101D2600A5E1B0E00E943416E05D0E946C140E94AA
:101D36009C13E05D0E946C140E944214E2E50E942E
:101D460068140E9429150E946E14E7ECF2E00E94C6
:101D5600CD13E9810E943B140E94F013E8810E9492
:101D66003B140E9471140E944E140E9409152CC245
:101D76000E945D16A091950BB091960B0E94591684
:101D860024F4A5E9BBE00E943A15E091950BF09189
:101D9600960B309719F4E0E0E093000510E012315D
:101DA60010F00C94200FA12FB0E0AF5FBF4F0E9440
:101DB6003416E13011F00C941E0F0E940A14E653FB
:101DC600F04F0081E12FE695E695E6952E2FE12F5F
:101DD600E770EF5F5E2FE22FF0E0EE56F44F1080D3
:101DE600E52F0E941515A12DB0E0EA23FB233097BD
:101DF600B9F40A3821F40E946D04E03009F406C0F3
:101E0600E12FEF5FEA93E0E0EA9380DF003810F01D
:101E16000B3808F001C00F5F003209F400E806C075
:101E2600003208F40F5F013808F000E00E940A143F
:101E3600E653F04F00831F5FB2CFE0E0F0E0E0939F
:101E4600DC0FF093DD0FE093E40C00E0003110F0BE
:101E56000C94EB0FE02F0E943515E03031F0AFEC1B
:101E6600BBE00E944015E07809F0B0C0E091E40CB8
:101E7600EF5FE093E40CAFEDBBE00E944015E0306D
:101E860079F40E9445150E941F150E943A150E947A
:101E960045150E94F413309711F40E944A158CC020
:101EA600E13011F00C94BB0F0E945015E1501E2F2B
:101EB6000E940A14E058F44FE081E030A9F40E9431
:101EC60053150E94B0130E945815309749F00E948E
:101ED60053150D901C900E945815E015F1050CF055
:101EE60002C00E944A151BC00E9445150E945D153E
:101EF600BF010E9445150E94F413DF010E940A14D7
:101F06000E9462150E94B613DB01ED93FC930E94BA
:101F16000A140E9467150E9453150E9424150E94F8
:101F260045150E94F413FF2332F40E9445150E94C2
:101F36001F150E9424150E9445150E94F413309720
:101F460011F40E944A150E946C150E94F4133097F2
:101F560071F00E946C150E941F150E943A150E948E
:101F66006C150E94F413309711F40E944A1524C090
:101F7600E23011F50E945015E1501E2F0E94711596
:101F86000E945D150F010E9471150E94F413DF0176
:101F96000E940A140E946215EA0FFB1FD001ED93FE
:101FA600FC930E940A140E946715AFE4BCE0E02F80
:101FB6000E9476150E94B0130E945015EA9316DE11
:101FC600AFEFBBE00E944015EA9310DE0F5F3ECFF5
:101FD600E091DC0FF091DD0FE093DF0CF093E00C65
:101FE60096C10E945F1630E010E0103168F40E943E
:101FF6000A14E156F44FE081AE2FEC81EA1711F492
:1020060031E002C01F5FF1CF303071F410E01031C3
:1020160058F40E940A14E156F44FE081E03011F4BE
:1020260031E002C01F5FF3CF313011F00C94B810CD
:10203600A091E20CA130A1F0E0919B0BF0919C0BDA
:10204600309721F4E0E00E94661663C1AFEDBBE075
:102056000E940A14EA0FFB1FA091990BA08307C0E8
:10206600AFEDBBE0EE27A10FBE1FE2E0EC93A0911F
:10207600970BA13118F0E0E0E093970BA091980B35
:10208600A13118F0E0E0E093980BAFEEBBE00E94C0
:102096000A14EA0FFB1FA091970BA083AFEFBBE0DA
:1020A6000E940A14EA0FFB1FA091980BA083AFEEC3
:1020B600BBE0EE27A10FBE1F2C91213068F0E22F66
:1020C600E150F0E00E946715E22FE150A6EABFE07A
:1020D6000E9476150E942415AFE0BCE00E940A1407
:1020E6000E945D15A0919B0BB0919C0BA083B183C0
:1020F600AFE2BCE00E940A140E945D15A0919D0B00
:10210600B0919E0BA083B1830E940A14E156F44F4E
:10211600AC81A083AFEBBBE00E940A14EA0FFB1F61
:10212600A091E70CA083AFECBBE00E940A14EA0F73
:10213600FB1FAD81A083AFE4BCE00E940A140E949D
:102146001F150E942415AFE6BCE00E940A140E94E7
:102156001F150E942415AFEABBE00E940A14EA0F7D
:10216600FB1FA0919A0BA08331E0E32F0E94661615
:10217600D0C01A9310E0103488F4E12FAFE9BBE029
:102186000E9476150E942415AFE1BCE00E940A1455
:102196000E941F150E9424151F5FEDCF10E012311B
:1021A60030F40E940A140E9467151F5FF8CFE98178
:1021B600E03009F406C0A091E30CAF5FE3E00E94B3
:1021C600FD15E093E30C18812296089524DD0C9406
:1021D600B9111A930A93E091E20CA091E10CEA1767
:1021E60089F00091E10C073009F415DD013019F48E
:1021F600E0E0EA93BEDF023019F4E1E0EA93E6DFBD
:102206000093E20CA091E20CA73019F4E0E0E09311
:102216007F0BA091E20CA13019F4E0E0E0937F0B74
:10222600A091E20CA23071F4A0910005A13020F03B
:10223600A091E60CAA230AF402C0E1E001C0E0E0A6
:10224600E0937F0B0991199108950E945D16E7E0CE
:10225600E093E10C10E0153110F00C948A110E9405
:102266000A140E942D1432960E9420169F010E9485
:102276000A140E942D1432960E942016AF010E9465
:102286000A140E942D143496E491E03011F0E130E6
:10229600B1F4D9010E943416AE2F0E940A140E948E
:1022A6002D143596E491EA1748F40E940A140E9408
:1022B6002D143696E491D9010E94481626C0E230C4
:1022C600A1F4DA010E943016E031A7E2FA0714F40D
:1022D600FF2352F40E940A140E942D1436960E947F
:1022E6002016DA010E94401610C0E33071F4D901BD
:1022F6000E943416EF3F49F40E940A140E942D14DE
:102306003696E491D9010E9448161F5FA4CF0E9419
:10231600641626960895E991F991A991B9911D90AF
:102326000590011421F40020D1F7EE270895101826
:10233600E1F3E1E008F4E2500895A991B991EE279E
:10234600FF276D91662311F03196FBCF0895AA27DA
:10235600BB27E991F9910590002011F01196FBCF6A
:10236600FD0108955D9BFECFE881ECB921960895A5
:102376001A930A93AC81BD810E941C163097C1F056
:10238600AA81BB810E941C168F01309749F002304A
:10239600E0E01E0760F0F80131978F01ED93FC93A2
:1023A600AC81BD810E94B0133197AE81A08303C07A
:1023B600EE81EA93D7DF198108812796089526973B
:1023C6000E945D1610E0EA89FB893196EA8BFB8B49
:1023D6003197E4912E2FE03011F40C940E13E12F77
:1023E600E03039F4253211F411E002C00E9478156C
:1023F60011C1E130A9F4253219F40E94781509C1FA
:1024060012E040E000E02D3211F401E003C12B326E
:1024160011F44BE2FFC0203211F440E2FBC002C0CF
:10242600E23039F450E013E0203311F40068F2C0D2
:1024360004C0E33011F00C940D13203310F02A334E
:1024460008F009C0A52FEAE0EA9FF0015E2FE22F0F
:10245600E0535E0FDFC0E22FE33649F40E94831596
:10246600E889F989A481AA930E948915D2C0E33725
:1024760041F40E9483150E9493150E94A0111E2FFD
:102486000AC0E03761F40E9483150E9493150E94EA
:10249600AA111E2F086002600F7730E035C0E436BF
:1024A60011F0E93611F4046002C0E53731F4E6E3D1
:1024B600F2E0EE83FF8315E00DC0E83511F4086005
:1024C60004C0E83711F00C940C13E0E4F2E0EE835C
:1024D600FF8314E002FF14C00E9483150E949D151D
:1024E600AB85AA233AF4EA85FB850E94B515EA87EF
:1024F600FB874DE2403011F01F5F01C00B7F04C027
:102506000E9483150E949D1500FD11C0151778F4D1
:1025160007FF08C002FF04C00B7F242F115001C023
:1025260020E301C020E20E9478155150EFCF312FF1
:1025360001FF1AC03030B9F003FF08C0EE81FF81F9
:102546003196EE83FF833197E49105C0AE81BF815A
:10255600ED91AE83BF83EA930E948915503009F04E
:1025660051503150E7CF4BC020E3EE81FF810E94EE
:102576002016E887F987EE81FF813296EE83FF8386
:10258600E885F985AA85BB85AE17BF0750F02F5F92
:10259600A885B985EA85FB85EA1BFB0BEA87FB87DD
:1025A600EFCF2A3328F003FF02C0295F01C0295D5F
:1025B60004FD1AC0213320F4A885B985119709F4C2
:1025C60009C0531710F000FF01C013C020E207FF37
:1025D6000BC020E3006102FF07C00B7F4A930E94F5
:1025E6008915503009F051500E947815503009F085
:1025F60051503150A885B985129708F0B5CF00FF24
:1026060008C0503031F05150E0E2EA930E9489153B
:10261600F8CF10E0D8CE0E94641664960895FF9213
:10262600F82E22971A930A93DE010E94B1158D01A6
:10263600DE0116960E94B1150E941C16EA83FB83E2
:10264600DE0114960E94B1150E941C16FA93EA93B5
:102656001A930A93FE013696FA93EA93E0E0F0E0C5
:10266600FA93EA93ACDEAA81BB81E0E0EC93198190
:1026760008812496FF900895E0E0EABBEFEFEBBBFC
:10268600E0916500EB7FE09365000895E0916500B9
:10269600E460E0936500E0E6E5BB08950A921A92CD
:1026A600FA926A937A938A939A93AA93BA93EA933D
:1026B600FA93EFB7EA930895E0915206EA930E94DF
:1026C6006304E09352060895EAE0F0E0FA93EA9391
:1026D6000895E0915206A3E4EA9FF0010895EB5FA6
:1026E600FA4FFA93EA930E94DC0CF3CFEE5FFA4FAF
:1026F600A0E0A083E1CFEA930E943104EA930C9410
:102706009704E8EEFCE0E093060DF093070D0895BC
:10271600A091060DB091070D0895A091060DB091F8
:10272600070D1796EC930895AF5FE4E60E94FD153A
:102736000895A0E0B0E00E9434160895E8ECF0E0B9
:10274600FA93EA930C94A515EA930E94A301E6E98D
:10275600F0E0FA93EA930C94A515ED91FD9131966C
:10276600FE93EE9308950E942916EA1BFB0B08952B
:10277600E881F981FA93EA930E946A0CECE2EA9303
:102786000C94380CFA93EA930E946A0CEBE3EA93F2
:102796000C94380CFA93EA930C94490CA0917B0B99
:1027A600B0917C0BAC910895A0917B0BB0917C0B02
:1027B600EC91EA930895ABE7BBE0CFCF0E940C0CF7
:1027C600E058FF4F1E2F0895E32FF0E00895EF77AE
:1027D600F0E0FA93EA930C946A0CEAE3EA930C9419
:1027E600380CEE0FFF1FAE0FBF1F0E941C16089578
:1027F600FA93EA930C946A0CE156F44FA0E0A08396
:102806000895EAE3EA930E94C30BE1300895E12FAD
:10281600F0E00895EA0FFB1F0F01AFECBBE0EE27D7
:10282600A30FBE1FEC910895F0E0FA93EA930E947D
:10283600760CD3CFA091790BB0917A0BE0E0EC93B4
:102846000E94641608950F01A0917B0BB0917C0B3A
:10285600EC9108950E94B915EA56FF4F0895EEE5EA
:10286600FBE0FA93EA930895E0915B0BF0E0F2CF78
:10287600F0E0BECF32960E942016DF010895A091A7
:10288600790BB0917A0B0895E0E6FAE0E0937B0BC2
:10289600F0937C0B0895E0915106A3E4EA9FF001C2
:1028A6000895EB5FFA4FE093790BF0937A0BE09182
:1028B6005C0AE5DFEC93A9E7BBE04FCFE0915B0A4A
:1028C600DEDFEC93A9E7BBE048CFEC93A9E7BBE0DA
:1028D60044CFD5DFFACFD3DFEFE0F7CFD0DFE0E0AC
:1028E600EC930895EE5FFA4FA1E0A083E0915106C4
:1028F600EA930E946304E0935106E1E00895E093B1
:10290600790BF0937A0B0895E0937B0BF0937C0B95
:102916000895E0917B0BF0917C0B0895A9E7BBE04D
:102926001CCFA0917B0BB0917C0B0895AA81BB8133
:10293600EC91E295E07FAE2FEC810895EA0FAA8133
:10294600BB81EC93A881B981EC91EF5F0895E12FEB
:10295600A091140DEA0FE093140D0895E091130D64
:10296600F0E0E55AF74F10830895E091130DEF5FFD
:10297600E093130D0895E091130DF0E0E55AF74F3B
:10298600A0E0A0830895F0E0E55AF74F0895E0919E
:102996007C0EF0917D0E0895A0917A0EB0917B0E7B
:1029A600EA17FB070895E12FA0910D0DEA0FE093BA
:1029B6000D0D0895E0910C0DF0E0E55AF54F1083EA
:1029C6000895E091810FF0E0E058F14FE081E09347
:1029D6009C00E091810FEF5FE093810F0895F0E096
:1029E600E030A1E0FA070895E12FA981BA81F0E06D
:1029F600EA0FFB1FE49108950E94C5150E94241654
:102A060084E00E94121328960C94560CEE5FFA4F3F
:102A1600A1E0A083E0915106EA930E946304E0934B
:102A260051060895A6E4B1E0F0E0EE0FFF1FEA0FAD
:102A3600FB1F0E9420160895EE0FFF1FAE0FBF1F4B
:102A46000895E0E0F0E0ED93FC930895E0915606DA
:102A5600E05D15DFEC93E0915606EF5FE770E093DB
:102A660056065CCFF0E0E156F44FE0810895ED9113
:102A7600FD913197FE93EE930895EE27A00FBE1FAA
:102A8600EC910895AFE0BCE0E02FF0E008950A93E2
:102A96000E94570EE02FF0E0AFCEAFEEBBE0EDCFD9
:102AA600E12FA6EABFE0F0E0C7CFE12FA2E8BFE042
:102AB600F0E097CEEE0FFF1FEA0FFB1F0895E058D8
:102AC600F44FE081F0E00895E058F44FA0E0A083D1
:102AD6000895AFE2BCE0E02FF0E00895AFE6BCE079
:102AE600E02FF0E00895F0E0A7CF2A93EF85F8896C
:102AF600FA93EA93FE013F96FA93EA930C94BB117C
:102B0600E889F9893497E88BF98B0895EF85F88978
:102B1600FA93EA93FE013F96FA93EA930C94BB115B
:102B2600A889B98914960E941C16EE83FF83FA932E
:102B3600EA930895A889B98914960E941C16EA8713
:102B4600FB870895E991F991309639F080EA9FE084
:102B56000197F1F7A8953197C9F708950024AF0DAD
:102B6600B01D0895F195E195F0400895EE0FFF1F11
:102B7600EE0FFF1FEE0FFF1F0895EF2FFF27E7FD54
:102B8600FFEF08956F2F660F660B762F0895FA9F55
:102B9600F02DEB9FF00DEA9FE02DF10D08953BD04F
:102BA600F6DF0EF4DFDF0895002498E0AA0F001C7C
:102BB6000E1A10F40E0E01C0A1609A95B9F7EA2F0D
:102BC600A02D08950024112490E1AA0FBB1F001C1C
:102BD600111C0E1A1F0A18F40E0E1F1E01C0A1604A
:102BE6009A9599F7FD01D001089515D0EBDF0EF403
:102BF600B9DF0895D9DFEA2F0895E894B7FF04C036
:102C0600A095B09511966894F7FDACDFDBDFFD016A
:102C16000EF4A8DF0895E894F7FF02C0A3DF6894D6
:102C2600B7FF06C0A095B095119600F8039400FA78
:102C36000895ED91FC91119708950590F491E02D7A
:102C460008957A936A93FA93EA9308951B2EBF2FF9
:102C5600F12D1A2EAE2FE12D0895119602D0FE2FDA
:102C66001197E199FECFFF93FFB7F894AEBBBFBBB8
:102C7600E09AEDB3FFBFFF91089507D01196EF9349
:102C8600EF2F03D0EF9111970895E19B02C0A8950D
:102C9600FCCF9FB7F894AEBBBFBBE09A8DB3E817E5
:102CA60019F0EDBBE29AE19A9FBF089500240A1637
:102CB6000B0608955A934A933A932A931A930A93C2
:102CC60008955D814C813B812A811981088108958F
:00000001FF
